:0200000480007A
:100000006F008004732F2034930F80006308FF0378
:10001000930F90006304FF03930FB0006300FF038E
:10002000130F000063040F0067000F00732F2034CC
:1000300063540F006F00400093E19153171F0000BD
:1000400023223FFC6FF09FFF93000000130100008C
:10005000930100001302000093020000130300004C
:100060009303000013040000930400001305000034
:10007000930500001306000093060000130700001C
:100080009307000013080000930800001309000004
:1000900093090000130A0000930A0000130B0000EC
:1000A000930B0000130C0000930C0000130D0000D4
:1000B000930D0000130E0000930E0000130F0000BC
:1000C000930F0000732540F16310050097020000B4
:1000D000938202017390523073500018970200000F
:1000E00093824202739052309B021000939252030B
:1000F0009382F2FF7390023B9302F0017390023AF5
:100100007350403097020000938242017390523046
:10011000735020307350303093010000970200007C
:10012000938282EE73905230130510001315F5017F
:10013000635C05000F00F00F930110009308D005D9
:10014000130500007300000093020000638A0200A0
:1001500073905210B7B200009B82921073902230BD
:100160007350003097020000938242017390123462
:10017000732540F17300203093000000130100004C
:1001800033A72002930300009301200063107746F9
:10019000930010001301100033A720029303000006
:1001A0009301300063147744930030001301700012
:1001B00033A72002930300009301400063187742A5
:1001C000930000003781FFFF33A720029303000054
:1001D00093015000631C7740B700008013010000BA
:1001E00033A720029303000093016000631077405F
:1001F000B70000803781FFFF33A72002B7030080DC
:10020000930170006314773E9B00D000939000022E
:100210001B01B00013110102B3A020029303F008E8
:10022000930180006394703C9B00700093901002D7
:100230001B01B0001311010233A120029303A00996
:10024000930190006314713A9B00D00093900002D8
:10025000B3A010029303900A9301A0006398703832
:10026000130200009B00D000939000021B01B0001D
:100270001311010233A72002130307001302120017
:1002800093022000E31052FE9303F0089301B000A4
:10029000631E7334130200009B00700093901002E1
:1002A0001B01B0001311010233A72002130000004C
:1002B000130307001302120093022000E31E52FCF6
:1002C0009303A0099301C00063127332130200006C
:1002D0009B00F000939000021B01B000131101027B
:1002E00033A72002130000001300000013030700CF
:1002F0001302120093022000E31C52FC9303500AE5
:100300009301D0006314732E130200009B00D000F1
:10031000939000021B01B0001311010233A72002C9
:100320001302120093022000E31252FE9303F0081E
:100330009301E000631C772A130200009B00700009
:10034000939010021B01B000131101021300000072
:1003500033A720021302120093022000E31052FE82
:100360009303A0099301F0006312772813020000A1
:100370009B00F000939000021B01B00013110102DA
:10038000130000001300000033A720021302120024
:1003900093022000E31E52FC9303500A93010001D4
:1003A00063167724130200009B00D0009390000294
:1003B000130000001B01B0001311010233A720023B
:1003C0001302120093022000E31052FE9303F00880
:1003D00093011001631C7720130200009B00700042
:1003E00093901002130000001B01B00013110102D2
:1003F0001300000033A72002130212009302200012
:10040000E31E52FC9303A009930120016310771EA1
:10041000130200009B00F000939000021300000004
:10042000130000001B01B0001311010233A72002CA
:100430001302120093022000E31E52FC9303500AA1
:10044000930130016314771A130200001B01B000FE
:10045000131101029B00D0009390000233A72002E9
:100460001302120093022000E31252FE9303F008DD
:1004700093014001631C7716130200001B01B000BA
:10048000131101029B0070009390100213000000F2
:1004900033A720021302120093022000E31052FE41
:1004A0009303A00993015001631277141302000013
:1004B0001B01B000131101029B00F0009390000299
:1004C000130000001300000033A7200213021200E3
:1004D00093022000E31E52FC9303500A9301600133
:1004E00063167710130200001B01B0001311010204
:1004F000130000009B00D0009390000233A720025D
:100500001302120093022000E31052FE9303F0083E
:1005100093017001631C770C130200001B01B000F3
:1005200013110102130000009B0070009390100251
:100530001300000033A720021302120093022000D0
:10054000E31E52FC9303A009930180016310770A14
:10055000130200001B01B000131101021300000080
:10056000130000009B00F0009390000233A72002CC
:100570001302120093022000E31E52FC9303500A60
:1005800093019001631477069B00F00193900002A1
:1005900033211002930300009301A001631871043A
:1005A0009B0010009390500233A1000293030000BF
:1005B0009301B001631C7102B32000029303000099
:1005C0009301C001639470029B001002939000029B
:1005D0001B0110011311110233A02002930300002C
:1005E0009301D00163147000631030020F00F00F0C
:1005F000638001009391110093E111009308D005ED
:1006000013850100730000000F00F00F930110002C
:100610009308D0051305000073000000731000C09C
:1006200000000000000000000000000000000000CA
:0C063000000000000000000000000000BE
:1010000000000000000000000000000000000000E0
:1010100000000000000000000000000000000000D0
:1010200000000000000000000000000000000000C0
:1010300000000000000000000000000000000000B0
:081040000000000000000000A8
:040000058000000077
:00000001FF
